:020000040800F2
:1000000000040024A1020008710F0008750F000809
:10001000C50F0008750F00089D0F0008A302000817
:10002000A3020008A3020008A3020008F1260008AA
:10003000A3020008A3020008A3020008A30200080C
:10004000A3020008A3020008A3020008A3020008FC
:10005000A3020008A3020008253C0008513C000848
:100060007D3C0008A93C0008D53C0008A30200081C
:10007000A3020008A3020008A3020008A3020008CC
:10008000A3020008A3020008A3020008A3020008BC
:10009000A3020008A3020008A3020008013D000813
:1000A000A3020008A3020008A3020008A30200089C
:1000B000A5380008A3020008A3020008A302000854
:1000C000A3020008A3020008A3020008A30200087C
:1000D000A3020008A3020008A3020008A30200086C
:1000E000693D0008A3020008A3020008A30200085B
:1000F000A3020008A3020008A3020008A30200084C
:10010000A3020008A3020008A3020008A30200083B
:10011000A3020008A3020008A3020008A30200082B
:10012000A3020008A3020008A3020008A30200081B
:10013000A3020008A3020008A3020008A30200080B
:10014000A3020008A3020008A3020008A3020008FB
:10015000A3020008A3020008A3020008A3020008EB
:10016000A3020008A3020008A3020008A3020008DB
:10017000A302000829320008A3020008A302000815
:10018000A3020008A302000815100008A30200083B
:10019000A3020008A3020008A3020008A3020008AB
:1001A000A3020008A3020008A3020008A30200089B
:1001B000A3020008A3020008A3020008A30200088B
:1001C000A3020008A3020008A3020008A30200087B
:1001D000A302000815320008A3020008A3020008C9
:1001E000A3020008A3020008A3020008A30200085B
:1001F000A3020008A3020008A3020008A30200084B
:10020000A3020008A3020008A3020008A30200083A
:10021000A3020008A3020008A3020008A30200082A
:10022000A3020008A3020008A3020008A30200081A
:10023000A3020008A3020008A3020008A30200080A
:10024000A3020008A3020008A3020008A3020008FA
:10025000A3020008A3020008A3020008A3020008EA
:10026000A3020008A3020008A3020008A3020008DA
:10027000A3020008A3020008A3020008A3020008CA
:10028000A3020008A3020008A3020008A3020008BA
:10029000A3020008A3020008A3020008A3020008AA
:1002A00002E000F000F8FEE772B6394880F30888F3
:1002B000384880F3098838484EF60851CEF20001DC
:1002C000086040F20000CCF200004EF63471CEF22D
:1002D00000010860BFF34F8FBFF36F8F40F2000043
:1002E000C0F2F0004EF68851CEF200010860BFF374
:1002F0004F8FBFF36F8F4FF00000E1EE100A4EF604
:100300003C71CEF200010860062080F31488BFF330
:100310006F8F02F02BFA03F045FA4FF055301F496A
:100320001B4A91423CBF41F8040BFAE71C49194AA9
:1003300091423CBF41F8040BFAE71A491A4A1B4B99
:100340009A423EBF51F8040B42F8040BF8E7002034
:100350001749184A91423CBF41F8040BFAE702F0F2
:1003600049FA03F093FA144C144DAC4203DA54F8F2
:10037000041B8847F9E700F041F8114C114DAC42DD
:1003800003DA54F8041B8847F9E702F031BA000099
:1003900000040024002400240000000800000024C1
:1003A00000040024C841000800240024382400244C
:1003B0003824002450390024A0020008A0020008BC
:1003C000A0020008A00200082DE9F04F2DED108AD0
:1003D000C1F80CD0D0F80CD0BDEC108ABDE8F08F7D
:1003E000002383F311882846A047002001F038FE3F
:1003F000FEE701F0E7FD00DFFEE7000038B51C4C2A
:100400006FF07403002523701E236570A570E570DE
:1004100025716571A571E57125726572A372E5722A
:1004200000F0E0FC20B10E2325726572A372E57224
:1004300002F040F90F4B984217D00133984241F235
:10044000883412BF002500240125002002F038F96D
:100450000DB100F0B5F800F02FFD00F047FC20468C
:1004600000F06EF900F0ACF8F9E700242546ECE75F
:1004700038240024010007B008B500F0B5FBA0F156
:1004800020035842584108BD07B5054B02211B887F
:10049000ADF8043001A800F013FC03B05DF804FBD4
:1004A000883E0008064991F8243033B10023082221
:1004B000086A81F8243000F03DBC0120704700BF7D
:1004C000582400242DE9F84F234C94F82430054695
:1004D000884617468BBB2E46DFF87C90002F38D01D
:1004E00094F824A0BAF1000F05D12022FF2148463C
:1004F000266200F0CFFCCAF10805BD4228BF3D4688
:100500005FFA85FBAD0041462A4604EB8A0000F005
:1005100097FC94F82430A7EB0B079B445FFA8BFB06
:10052000BBF1080F2E44A844FFB284F824B0D5D103
:10053000FFF7B8FF0028D1D108E0266A06EB830652
:10054000B042C9D0FFF7AEFF0028C4D10020BDE8FB
:10055000F88F0120BDE8F88F5824002410B520231F
:1005600083F311881248C3680BB101F0FFFD00232B
:10057000104A0F484FF47A7101F0BCFD002383F359
:1005800011880D4C236813B12368013B2360636815
:1005900013B16368013B6360084B1B7833B9636830
:1005A00023B9022000F03AFC3223636010BD00BF83
:1005B000442400245D0500088829002480240024A8
:1005C0002DE9F041544B554953F8042F013201D124
:1005D000BDE8F0818B42F7D1514C524B22689A42D0
:1005E00040F29880504B9B6803F1006303F50033A1
:1005F0009A4280F08F80002000F094FB4B4B022049
:10060000187000F0FFFB4A4BD3F8E8200022C3F833
:10061000E820D3F81011C3F81021D3F81011D3F843
:10062000EC10C3F8EC20D3F81411C3F81421D3F85C
:100630001411D3F8F010C3F8F020D3F81811C3F850
:100640001821D3F81811D3F8801041F00061C3F8D5
:100650008010D3F8801021F00061C3F88010D3F827
:100660008010D3F8801041F00071C3F88010D3F8E7
:10067000801021F00071C3F88010D3F8803072B67A
:100680002C492D4B0B601D682468BFF34F8FBFF3BF
:100690006F8F2A4BC3F88420BFF34F8F5A6922F41F
:1006A00080325A61BFF34F8FD3F88020C2F3C9065E
:1006B000C2F34E325201B70743F6E07E02EA0E085B
:1006C00038463146013948EA000CB1F1FF3FC3F822
:1006D00074C200F14040F5D1203A12F1200FEDD163
:1006E000BFF34F8FBFF36F8FBFF34F8FBFF36F8F8A
:1006F0005A6922F400325A610022C3F85022BFF333
:100700004F8FBFF36F8F202383F31188AD4685F39E
:1007100008882047BDE8F081FCFF01081C000208A2
:1007200004000208FFFF010838240024802400246C
:100730000044025808ED00E00000020800ED00E06F
:100740002DE9F04FB54C97B020228246FF210EA82C
:10075000A56800F09FFBB24A1378A046A3B9B14840
:100760000121C3601170202383F31188C3680BB18A
:1007700001F0FCFC0023AC4AAA484FF47A7101F066
:10078000B9FC002383F31188DFF8BCB2BAF1000F83
:1007900001D0CBF800A0A54F00243C70CBF804405A
:1007A0002646012000F02EFBBAF1000F00F0E08198
:1007B000DBF80030002B40F0DB8117B0BDE8F08F94
:1007C0000220FFF759FE002840F0D081984B1B888B
:1007D000ADF82430022109A800F072FAE1E74FF4E5
:1007E0007A7000F001FA031E0193EFDB0220FFF79D
:1007F00043FE81460028E9D0019B581E0428E5D815
:10080000DFE800F0030C0F12150016A8052340F8CE
:10081000343D042100F054FA4C4650E004217F4856
:10082000F8E704218348F5E704218348F2E71C2414
:10083000204600F079FA04340990042109A800F058
:100840003FFA2C2CF4D1E7E7002EBFD0002CBDD00E
:100850000220FFF711FE064610B901242646B5E72F
:10086000012000F05FFA0220387000F0CBFA00247B
:10087000E3B21846019300F065FA814648B1019B46
:10088000184600F06FFA01340028F1D134466B4B62
:100890009DE7012302203B7000F0A6FA4D46D8F8F0
:1008A00008309D4206D2284600F03EFA0130EDD1D4
:1008B0000435F4E700253D70CBF80450344600F0D1
:1008C000F1FAFFF7E1FD4EE1002E3FF47FAF002C7F
:1008D0003FF47CAF0220387000F094FA322000F030
:1008E00083F9041EB9DB14F00306B6D1D8F808204A
:1008F0002B199342B1D8B4F5807FAED8DFF8409180
:10090000A6420CDA4FF47A7000F06EF90390039B64
:10091000002BA2DB039B06F809300136F0E7C82064
:10092000FFF7AAFD0646002897D01F2D11D8C5F164
:100930002009A14528BFA1460EAB25F003004A4679
:100940003F49184400F07CFA4A46FF213C4800F039
:10095000A1FA4FEAA4095FFA89F239492846FFF75C
:10096000B1FD0446002891D005EB89050646A6E7AF
:100970000220FFF781FD00283FF428AFFFF792FD2A
:1009800000283FF423AF4FF0000AD146D8F80830D2
:100990009A453CD2BAF11F0F1CD80E9B013319D0D7
:1009A0002AF0030316AA134453F8203C099325495F
:1009B0004B68A3B1002209A8135C83EA0903DBB2E8
:1009C000013251F82330042A83EA1929F4D10AF1BB
:1009D000040ADBE7504600F0A7F90990E7E71A465A
:1009E000082012F0010F4FEA52021FBF82F06D4241
:1009F00082F4380282F4034282F020020138F0D1FE
:100A000041F823200133B3F5807FE8D1D2E716A85F
:100A1000042140F8489D00F053F950E738240024A1
:100A200084250024442400245D050008802400243B
:100A30008A3E00083C240024402400248C3E000808
:100A400084240024882500248829002416A8002353
:100A500040F8343D642100F0FFF800287FF4B6AE82
:100A60000220FFF709FD00283FF4B0AE099800F01E
:100A70008BF916AB43F8440D04211846CBE716A8B2
:100A8000002340F8343D642100F0E6F800287FF4AC
:100A90009DAE0220FFF7F0FC00283FF497AE0998C6
:100AA00000F074F916AB43F8400DE5E70220FFF7BC
:100AB000E3FC00283FF48AAE00F06EF916AB43F871
:100AC0003C0DD9E70220FFF7D7FC00283FF47EAEAB
:100AD00009A9142000F066F9814616A8042140F8FF
:100AE000389D00F0EDF8494609A894E74FF47A7074
:100AF000FFF7C2FC00283FF469AEFFF7D3FC0028E3
:100B00003FF4C5AE0E9B01330CD008220EA9002085
:100B1000FFF7D8FC00283FF4BAAE2022FF210EA830
:100B200000F0B8F9FFF7B0FC2E4801F09FFA44E658
:100B300016A8002340F8343D642100F08DF8002809
:100B40007FF444AE0220FFF797FC00283FF43EAE4E
:100B5000FFF79AFC41F2883001F088FA099800F01A
:100B6000E7F900F09FF94FF0000A1AE60646A6E6FC
:100B7000002000F039F80390039B002BFFF614AE21
:100B8000012000F031F9039B213B122B3FF609AE07
:100B900001A252F823F000BFC1070008DF070008D8
:100BA00049080008A3070008A3070008A3070008D6
:100BB000C9080008A3070008710900084D0A0008C9
:100BC0007F0A0008AD0A0008A3070008C50A00084C
:100BD000A3070008ED0A0008BF080008A3070008E3
:100BE000310B0008A08601002DE9F34702AE002476
:100BF0004FF47A7506F8014D144FDFF858804543DD
:100C000097F900305A1C5FFA84F901D0A34212D13F
:100C100058F8240003680122D3F820A031462B465F
:100C2000D047012807D10A4B9DF8070083F80090B0
:100C300002B0BDE8F0870134022CE1D14FF4FA7024
:100C400001F014FA4FF0FF30F2E700BF0024002457
:100C5000AC290024903E00082DE9F0474FF47A7546
:100C6000144FDFF8588006464D43002497F90030B2
:100C70005A1C5FFA84F901D0A34210D158F824001D
:100C800003680422D3F820A031462B46D04704281D
:100C900005D1094B83F800900020BDE8F0870134AE
:100CA000022CE3D14FF4FA7001F0E0F94FF0FF307D
:100CB000BDE8F08700240024AC290024903E000801
:100CC00030B4074B1A78074B53F822402368DD698C
:100CD000054B0A46AC460146204630BC604700BF83
:100CE000AC290024903E0008A0860100F8B501F070
:100CF00005FC094C094E0A4F207000253068237806
:100D0000834207D901F0F6FB336805440133BD4245
:100D10003360F3D9F8BD00BFAD2900249029002429
:100D2000FFFF010001F0B2BC00F1006000F50030EF
:100D30000068704700F10060920000F5003001F09B
:100D400047BC0000054B1A68054B1B789B1A834271
:100D500002D9104401F0CEBB002070479029002436
:100D6000AD29002438B5074D04462868204401F019
:100D7000C7FB28B928682044BDE8384001F0D2BB41
:100D800038BD00BF9029002400207047014BC05897
:100D9000704700BF00E8F11F014B1868704700BFA3
:100DA0000010005C70B50E4B5C6893F90860013868
:100DB0000A18013C0B4693420FD214F9015F581CEC
:100DC0001DB1034600F8015CF5E72C2482421C703B
:100DD00001D9981C5E70401A70BD1846FBE700BF31
:100DE0000424002400207047022804D14FF400029C
:100DF000034B9A6170470128FCD14FF48002F7E75A
:100E000000080258022803D18022034B9A617047E0
:100E10000128FCD14022F8E700080258022805D139
:100E2000064A536983F08003536170470128FCD15F
:100E3000024A536983F04003F6E700BF00080258F6
:100E400010B50023934203D0CC5CC4540133F9E7BE
:100E500010BD000030B5441E14F9010F0B4660B1FF
:100E600093F90050854201F1010106D11AB993F9B5
:100E70000020801A30BD013AEEE7002AF7D1104673
:100E800030BD000002460346981A13F9011B0029E1
:100E9000FAD1704702440346934202D003F8011B83
:100EA000FAE77047024B1A78024B1A70704700BF7E
:100EB000AC2900240024002438B5174D174C2846CF
:100EC00000F006FC2146284600F02EFC236814485A
:100ED000D3F89020D2F8043843F00203C2F8043863
:100EE00001F0C4F80F49206800F02EFD23680E4879
:100EF000D3F890200D49D2F8043823F00203C2F849
:100F00000438A8424FF4E1330B6003D0BDE8384009
:100F100000F03CBB38BD00BF5C2E0024643F0008DD
:100F200040420F00B43F0008B02900249429002457
:100F300038B50B4B1A780B4B53F822400A4B9C42A6
:100F400005460CD0094B002118461822FFF7A2FFD6
:100F5000056001462046BDE8384000F017BB38BDAB
:100F6000AC290024903E00085C2E00249429002423
:100F7000FEE7000000B59BB0EFF3098168226846E8
:100F8000FFF75EFFEFF30583034B9A6B9A6A9A6A49
:100F90009A6A9A6A9B6AFEE700ED00E000B59BB092
:100FA000EFF3098168226846FFF74AFFEFF30583F4
:100FB000034B9A6A9A6A9A6A9A6A9A6A9B6AFEE7E5
:100FC00000ED00E000B59BB0EFF3098168226846B0
:100FD000FFF736FFEFF30583034B5A6B9A6A9A6A61
:100FE0009A6A9A6A9B6AFEE700ED00E0024A13687B
:100FF00043F0C0031360704700780040044B5A6808
:1010000010439A6858600AB1181D1047704700BF16
:10101000B02900242DE9F84F404EF56D2F68EC699A
:101020002C62210718D014F0080F0CBF002080207C
:10103000E20748BF40F02000A30748BF40F040004F
:10104000610748BF40F48070202383F31188FFF7C5
:10105000D5FF002383F31188E20509D5202383F30C
:1010600011884FF40070FFF7C9FF002383F3118844
:10107000DFF8A8A04FF020094FF0000B14F0200873
:1010800032D13B0615D5DFF898A04FF02009200695
:101090000FD589F31188504600F0ECF9002830DABA
:1010A0000820FFF7ABFF27F080032B60002383F3BA
:1010B000118879060DD562060BD5202383F311889C
:1010C000F26C336D9A4201D1336C03BB002383F37E
:1010D0001188E30604D5B26E13690BB150699847C5
:1010E000BDE8F84F01F014BB89F31188AB8C96F87A
:1010F00064105046194000F057FA8BF31188EC69E0
:10110000BCE780B2288588F31188EC69BFE710201E
:1011100027F04007FFF772FF2F60D7E7B0290024C0
:10112000E829002413B5104C204600F023FA04F1FE
:101130001400009400234FF400720C4900F0E4F80E
:1011400004F1380000940A4B0A494FF4007200F091
:101150005DF9094BE365094B23660C21522002B06F
:10116000BDE8104000F05EB8B02900241C2A00241D
:10117000ED0F00081C2C00240078004000366E01A2
:10118000254B002908BF1946037C8166012B30B529
:1011900011D1224B98420ED1214BD3F8E82042F0D6
:1011A0008042C3F8E820D3F8102142F08042C3F80F
:1011B0001021D3F810310A68036EC46D03EB52039B
:1011C000B3FBF2F34A68150442BF23F0070503F0AE
:1011D000070343EA4503E3608B6843F04003636021
:1011E000CB6843F00103A36042F4967343F001031C
:1011F000236051054FF0FF33236205D512F0102212
:1012000005D0B2F1805F04D080F8643030BD7F2318
:10121000FAE73F23F8E700BFA83E0008B029002402
:101220000044025800F1604300F01F02400903F53A
:10123000614309018000C9B200F1604083F80013E6
:1012400000F5614001239340C0F88031036070478E
:10125000F8B5154682680669AA420B46816938BF0F
:101260008568761AB542044607D218462A46FFF723
:10127000E7FDA3692B44A3610DE011D9324618465E
:10128000FFF7DEFDAF1B3A46E1683044FFF7D8FDBB
:10129000E2683A44A261A3685B1BA3602846F8BDDC
:1012A00018462A46FFF7CCFDE368E4E783682DE99A
:1012B000F041044693421546266938BF8568406967
:1012C000361AB5420F4606D22A46FFF7B9FD6369C2
:1012D0002B4463610DE012D93246A5EB0608FFF7F7
:1012E000AFFD4246B919E068FFF7AAFDE268424443
:1012F0006261A3685B1BA3602846BDE8F0812A46B3
:10130000FFF79EFDE368E4E710B50A440024C361DB
:10131000029B006040608460C16081614161026144
:10132000036210BD08B582694369934201D18268A6
:1013300082B98268013282605A1C42611970426926
:1013400003699A4201D3C3684361002100F0AAFEF9
:10135000002008BD4FF0FF3008BD000070B520230D
:1013600004460E4683F31188A568A5B1A368A26957
:10137000013BA360531CA36115782269934224BFEB
:10138000E368A361E3690BB120469847002383F328
:101390001188284670BD3146204600F073FE0028B3
:1013A000E2DA85F3118870BD2DE9F74F05460F4647
:1013B00090469A46D0F81C90202686F311884FF06C
:1013C000000B144664B1224639462846FFF740FF19
:1013D000034668B95146284600F054FE0028F1D073
:1013E000002383F31188A8EB040003B0BDE8F08F5D
:1013F000B9F1000F03D001902846C847019B8BF339
:101400001188E41A1F4486F31188DBE7C16081610B
:101410004161C3611144009B0060406082600161D2
:1014200003627047F8B504460E461746202383F33F
:101430001188A568A5B1A368013BA36063695A1C24
:1014400062611E70236962699A4224BFE368636126
:10145000E3690BB120469847002080F31188F8BD5E
:101460003946204600F00EFE0028E2DA85F31188A6
:10147000F8BD0000836942699A4210B501D18268C3
:101480007AB98268013282605A1C82611C780369D1
:101490009A4201D3C3688361002100F003FE204615
:1014A00010BD4FF0FF3010BD2DE9F74F05460F4638
:1014B00090469A46D0F81C90202686F311884FF06B
:1014C000000B144664B1224639462846FFF7EEFE6B
:1014D000034668B95146284600F0D4FD0028F1D0F3
:1014E000002383F31188A8EB040003B0BDE8F08F5C
:1014F000B9F1000F03D001902846C847019B8BF338
:101500001188E41A1F4486F31188DBE702684368F8
:101510001143016003B11847704700001430FFF712
:1015200043BF00004FF0FF331430FFF73DBF000012
:101530003830FFF7B9BF00004FF0FF333830FFF706
:10154000B3BF00001430FFF709BF00004FF0FF31B8
:101550001430FFF703BF00003830FFF763BF00000F
:101560004FF0FF323830FFF75DBF000000207047BA
:10157000FFF7D8BD044B0360002343608360C36062
:1015800001230374704700BFC03E000810B520233C
:10159000044683F31188FFF7F3FD0223237400232D
:1015A00083F3118810BD000038B5C36904460D46A9
:1015B0001BB904210844FFF7A9FF294604F11400D0
:1015C000FFF7B0FE002806DA201D4FF48061BDE869
:1015D0003840FFF79BBF38BD026843681143016084
:1015E00003B118477047000013B5446BD4F8943426
:1015F0001A681178042915D1217C022912D1197990
:10160000128901238B4013420CD101A904F14C0033
:1016100001F03CFFD4F89444019B217902462068F4
:1016200000F0EAF902B010BD143001F0BFBE0000B6
:101630004FF0FF33143001F0B9BE00004C3001F020
:1016400091BF00004FF0FF334C3001F08BBF000022
:10165000143001F08DBE00004FF0FF31143001F066
:1016600087BE00004C3001F05DBF00004FF0FF323C
:101670004C3001F057BF0000D0F8942438B51368FF
:1016800019780429054601D0012038BD017C0229C2
:10169000FAD112795C89012090400440F4D105F11F
:1016A000140001F01FFE02460028EDD0D5F8945436
:1016B0004FF480732868697900F08CF9204638BDB2
:1016C000406BFFF7D9BF0000002070477047000053
:1016D0007FB5124B0360002343608360C360012524
:1016E00002260F4B057404460290019300F1840218
:1016F000294600964FF48073143001F0CFFD094B5A
:101700000193029400964FF4807304F523722946E6
:1017100004F14C0001F096FE04B070BDE83E0008F4
:10172000C1160008E91500080A68202383F3118810
:101730000B790B3342F823004B79133342F8230023
:101740008B7913B10B3342F8230002230374C0F8E2
:101750009414002383F311887047000038B5037F89
:10176000044613B190F85430ABB9201D0125022175
:10177000FFF732FF04F1140025776FF0010100F04C
:101780009DFC84F8545004F14C006FF00101BDE859
:10179000384000F093BC38BD10B501210446043038
:1017A000FFF71AFF0023237784F8543010BD0000A0
:1017B00038B504460025143001F088FD04F14C00D2
:1017C000257701F057FE201D84F854500121FFF7C2
:1017D00003FF2046BDE83840FFF74EBF90F8803049
:1017E00003F06003202B19D190F88120212A0AD020
:1017F000222A4FF000030ED0202A0FD1084A426758
:101800000722826704E0064B4367072383670023B0
:10181000C3670120704743678367F9E7002070477B
:1018200010240024D0F8943437B51A6811780429AC
:1018300004461AD1017C022917D119791289012392
:101840008B40134211D100F14C05284601F0D2FE25
:1018500058B101A9284601F019FED4F89444019B1F
:1018600021790246206800F0C7F803B030BD0000BF
:1018700001F10B03F7B550F8234005460E46F4B1CD
:10188000202383F3118805EB8607201D0821FFF72D
:10189000A3FEFB685B691B684C3413B1204601F062
:1018A00003FE01A9204601F0F1FD024648B1019B6B
:1018B0003146284600F0A0F8002383F3118803B0D6
:1018C000F0BDFB685A691268002AF5D01B8A013BFB
:1018D0001340F1D105F18002EAE70000133138B579
:1018E00050F82140DCB1202383F31188D4F89424EC
:1018F0001368527903EB8203DB689B695D6845B12D
:1019000004216018FFF768FE294604F1140001F075
:10191000F3FC2046FFF7B0FE002383F3118838BDA7
:101920007047000000F0EEBF012303700023436006
:1019300000F1300200F1500142F8043B8A42D361C9
:10194000FAD103814381704738B50446202383F3DD
:1019500011880025416000F10C0300F1300243F8CA
:10196000045B9342FBD1204600F0EEFF022323707C
:1019700085F3118838BD000070B500EB8103054682
:101980005069DA600E46144618B110220021FFF7A4
:1019900081FAA06918B110220021FFF77BFA3146C5
:1019A0002846BDE8704001F0E1B80000038903F06B
:1019B00001030381438903F00103438100F13002F5
:1019C00000F11003002143F8041B9342FBD101F006
:1019D00065B90000F0B400EB81044789E468012593
:1019E000A4698D403D43458123600023A26063606C
:1019F000F0BC01F081B90000F0B400EB810407896C
:101A0000E468012564698D403D430581236000231E
:101A1000A2606360F0BC01F0F9B90000022310B5C8
:101A2000037000230446A0F8883080F88A3080F8DC
:101A30008B300381438100F10C0200F1300142F848
:101A4000043B8A42FBD184F87030204601F022F832
:101A500063681B6823B120460021BDE81040184789
:101A600010BD0000436802781B6880F88C200522B6
:101A700002700BB10421184770470000436890F8CA
:101A80008C201B6802700BB10521184770470000BD
:101A900090F8703070B5044613B1002380F87030B0
:101AA00004F18002204601F01DF963689B6863BB66
:101AB00094F8805015F0600615D194F8813005F047
:101AC0007F0545EA032540F202339D4200F00E8176
:101AD0005BD8022D00F0DC803FD8002D00F087801D
:101AE000012D00F0CF800021204601F0B3FB002142
:101AF000204601F0A3FB63681B6813B10621204652
:101B00009847062384F8703070BD20469847002817
:101B1000CED094F8872094F8863043EA0223A26F4F
:101B2000934238BFA36794F98030A56F002B4FF024
:101B3000200380F2FD80002D00F0EC80092284F863
:101B4000702083F311880021A36F626F2046FFF796
:101B500053FF002383F3118870BDB5F5817F00F03A
:101B6000B180B5F5407F49D0B5F5807FBBD194F801
:101B70008230012BB7D1B4F8883023F00203A4F8E7
:101B800088306667A667E667C3E740F201639D4257
:101B90001ED8B5F5C06F3BD2B5F5A06FA3D1B4F890
:101BA0008030B3F5A06F0ED194F8823084F88A307B
:101BB000204600F0CDFF63681B6813B10121204669
:101BC00098470323237000236367A367E367A0E7B5
:101BD000B5F5106F32D040F602439D4252D0B5F5B4
:101BE000006F80D104F18B036367012324E004F1CB
:101BF000880363670223A367E5678AE794F8823066
:101C0000012B7FF470AFB4F8883043F00203B6E7DD
:101C100094F88520616894F884304D6894F88310B6
:101C200043EA0223204694F88220A84700283FF484
:101C30005AAF436863670368A367A4E72378042B5C
:101C400010D1202383F311882046FFF7AFFE86F3DF
:101C50001188636884F88B601B68032121700BB1C5
:101C60002046984794F88230002BACD084F88B3013
:101C70000423237063681B68002BA4D00221204634
:101C80009847A0E7374B63670223A36700239DE7CC
:101C900094F8841011F0800F204601F00F010ED04F
:101CA00001F012F8012806D002287FF41CAF2E4B59
:101CB0006367A06767E72D4B6367A56763E700F07D
:101CC000F5FFEFE794F88230002B7FF40CAF94F827
:101CD000843013F00F013FF476AF1A06204602D588
:101CE00001F0D0FA6FE701F0C1FA6CE794F88230A6
:101CF000002B7FF4F8AE94F8843013F00F013FF41A
:101D000062AF1B06204602D501F0A4FA5BE701F0A2
:101D100095FA58E7142284F8702083F311882B4633
:101D20002A4629462046FFF755FE85F3118870BDE7
:101D30005DB1152284F8702083F311880021A36F10
:101D4000626F2046FFF746FE03E70B2284F87020FF
:101D500083F311882B462A4629462046FFF74CFE7E
:101D6000E3E700BF183F0008103F0008143F0008D9
:101D700038B590F870300446152B29D8DFE803F009
:101D80003E28282828283E28280B293928282828B2
:101D9000282828283E3E90F8871090F88620836FE8
:101DA00042EA01229A4214D9C268128AB3FBF2F5C0
:101DB00002FB15356DB9202383F311882B462A4683
:101DC0002946FFF719FE85F311880A2384F870303D
:101DD00038BD142384F87030202383F31188002346
:101DE0001A4619462046FFF7F5FD002383F31188B4
:101DF00038BDC36F03B198470023E7E7002101F026
:101E000029FA0021204601F019FA63681B6813B112
:101E10000621204698470623D8E7000090F8702056
:101E2000152A38B5044622D80123934040F6416272
:101E300013421DD113F480150FD19B0217D50B232C
:101E400080F87030202383F311882B462A462946D8
:101E5000FFF7D2FD85F3118838BDC3689B695B68C5
:101E60002BB9C36F03B19847002384F8703038BD95
:101E7000002101F0EFF90021204601F0DFF963684D
:101E80001B6813B10621204698470623EDE70000A2
:101E9000024B00221B605B609A6070471C2E00247E
:101EA000002303748268054B1B6899689142FBD23A
:101EB0005A68036042601060586070471C2E00240E
:101EC00008B5202383F31188037C032B05D0042B52
:101ED0000DD02BB983F3118808BD436900221A6025
:101EE0004FF0FF334361FFF7DBFF0023F2E790E899
:101EF0000C001A6002685360F2E7000000230374CC
:101F00008268054B1B6899689142FBD85A68036048
:101F100042601060586070471C2E0024054B196900
:101F20000874186802681A6053601861012303740A
:101F3000FEF74ABA1C2E002430B54B1C87B005466C
:101F40000A4C10D023690A4A01A800F0D3F82846A9
:101F5000FFF7E4FF049B13B101A800F007F9236920
:101F6000586907B030BDFFF7D9FFF8E71C2E0024F1
:101F7000C11E000838B50C4D41612B6981689A6813
:101F80009142044603D8BDE83840FFF789BF1846A0
:101F9000FFF786FF01232C61014623742046BDE82C
:101FA0003840FEF711BA00BF1C2E0024044B1A68FB
:101FB0001B6990689B68984294BF0020012070477D
:101FC0001C2E002410B5084C236820691A68226072
:101FD0005460012223611A74FFF790FF01462069C3
:101FE000BDE81040FEF7F0B91C2E002482600222EA
:101FF00002740022427470478368A3F17C0243F8A4
:102000000C2C026943F83C2C426943F8382C074AEF
:1020100043F81C2CC26843F8102C022203F8082C49
:10202000002203F8072CA3F118007047E103000811
:1020300010B5202383F31188FFF7DEFF002104464B
:10204000FFF798FF002383F31188204610BD00009E
:10205000024B1B6958610F20FFF760BF1C2E002444
:10206000202383F31188FFF7F3BF000008B5014672
:10207000202383F311880820FFF75EFF002383F3FA
:10208000118808BD49B1064B42681B6918605A6047
:10209000136043600420FFF74FBF4FF0FF307047DD
:1020A0001C2E00240368984206D01A680260506013
:1020B00059611846FFF7F4BE7047000038B5044672
:1020C0000D462068844200D138BD036823605C60FF
:1020D0004561FFF7E5FEF4E7054B03F114025A6191
:1020E0009A614FF0FF32DA6100221A62704700BF36
:1020F0001C2E0024F8B503614FF08043C2605C6A77
:10210000194B1A46022952F8145F38BF0221954232
:1021100006461F460AD1586198611C6205604560F9
:1021200081600819BDE8F84001F086BA186AAB680A
:10213000241A0C1902D3E41A2D6804E09C4202D23E
:10214000204401F087FAAB689C42F4D86B68736056
:1021500035601E606E60B460A9684FF0FF33091BE4
:10216000A960FB61F8BD00BF1C2E002410B41B4CFD
:10217000234653F8141F814210D0416802680A6058
:10218000026851609A424FF00001C16003D0936829
:1021900081680B4493605DF8044B70470A68626184
:1021A00000209A425360C86003D15DF8044B01F0EF
:1021B0004BBA93688868034493604FF08042206A6A
:1021C000526A121A9342E6D9991A012998BF931CB0
:1021D00018445DF8044B01F03DBA00BF1C2E0024EA
:1021E00000207047FEE70000704700004FF0FF300E
:1021F00070470000022906D0032906D001290648AD
:1022000018BF0020704705487047032A9ABF04484A
:1022100000EBC2000020704710400008C43F0008D7
:102220001824002470B5044608460D46FEF72AFE21
:10223000C6B22046013403780BB9184670BD324649
:102240002946FEF707FE0028F3D1012070BD0000EB
:102250002DE9F04F81469BB008460D461646FEF725
:1022600011FE3D49C4B22846FFF7DCFF08B1043433
:10227000E4B23A492846FFF7D5FF08B11034E4B27A
:10228000632C01AF0CD8DFF8E0A0DFF8E0B03C46EB
:1022900095F80080B8F1000F1CD184F8008003E0AD
:1022A0002946384601F0E8FD3846FEF7EBFDC0B29E
:1022B000431C5B0089E848003370032373700023DC
:1022C00002361946DAB2904206F102063DD81BB03A
:1022D000BDE8F08FB8F1250F32D107221E492846FC
:1022E000FEF7B8FD70B9DBF800202260DBF80420AF
:1022F0006260BBF8082022819BF80A20A272073591
:102300000B34C5E7082215492846FEF7A3FDB8B9E6
:102310001348A21C10F8011F124B4FEA111E01F0C6
:102320000F011EF80AE011F80A1002F802EC9842B8
:1023300002F8011C02F10202ECD118340835A7E7BB
:1023400084F8008001350134A2E7FA5C06F8022C1B
:1023500006F8011C0133B5E76C3F0008743F000824
:10236000FFE7F11F0BE8F11F893F00087D3F0008E0
:1023700008B5202383F311880348FFF753FA00239D
:1023800083F3118808BD00BF5C2E002410B50446FD
:10239000052916D8DFE801F016150316161D2023AF
:1023A00083F311880E4A0121FFF7E6FA20460D4A11
:1023B0000221FFF7E1FA0C48FFF7FAF9002383F353
:1023C000118810BD202383F311880748FFF7C6F951
:1023D000F4E7202383F311880348FFF7DDF9EDE7E5
:1023E0001C3F0008403F00085C2E002438B50C4D0F
:1023F0000C4C0D492A4604F10800FFF729FF05F1AE
:10240000CA0204F110000949FFF722FF05F5CA725C
:1024100004F118000649BDE83840FFF719BF00BFB6
:1024200024330024182400249C3F0008A63F000801
:10243000743F0008BFF34F8F044B1A695107FCD15A
:10244000D3F810215207F8D1704700BF0020005286
:1024500008B50D4B1B78ABB9FFF7ECFF0B4BDA68F7
:10246000D10741BF0A4A5A6002F188325A60D3F854
:102470000C21D20741BF064AC3F8042102F1883279
:10248000C3F8042108BD00BF82350024002000529B
:102490002301674508B5114B1B78F3B9104B1A6936
:1024A000510742BFDA6842F04002DA60D3F81021E7
:1024B000520742BFD3F80C2142F04002C3F80C216E
:1024C000FFF7B8FF064BDA6842F00102DA60D3F892
:1024D0000C2142F00102C3F80C2108BD8235002412
:1024E000002000520F289ABF00F5806040040020B1
:1024F000704700004FF40030704700001020704714
:102500000F2808B50BD8FFF7EDFF00F50033026880
:10251000013204D104308342F9D1012008BD0020EA
:1025200008BD00000F2810B504464AD8FFF782FF07
:10253000FFF78EFF24484FF0FF33072C4361C0F8AC
:10254000143124D80361FFF775FF230243F02403FD
:10255000C360C36843F08003C36003695A07FCD4B7
:10256000FFF768FF2046FFF7BDFF00F50033BFF31C
:102570004F8F164A984220D3BFF34F8FBFF36F8F10
:10258000FFF788FF2046BDE81040FFF7B9BFC0F84D
:102590001031FFF74FFFA4F108031B0243F024039F
:1025A000C0F80C31D0F80C3143F08003C0F80C3186
:1025B000D0F810315B07FBD4D2E7C2F85C022030C0
:1025C000D8E7002010BD00BF0020005200ED00E061
:1025D0002DE9F84F42EA0003DB0605460E46174692
:1025E00043D1FFF735FFDFF89880DFF89890DFF8E8
:1025F00098A034463B1B33441F2B04D8FFF74AFFF7
:102600000120BDE8F88F1C4A1C4805F1784393422D
:102610009ABF5046C346CB46FFF70CFF4FF0FF333F
:10262000CBF80030036843F00203036004F11C019F
:10263000231F53F804EFEA18121B8B42C2F800E084
:10264000F7D1BFF34F8FFFF7F5FE4FF0FF33CBF815
:102650000030036823F0020303602022214628464D
:1026600001F0FAFB20B1FFF715FF0020BDE8F88F5D
:1026700020352034BEE700BFFFFF0F000C210052C1
:1026800014200052142100520C20005210B5084CA6
:10269000237828B153B9FFF7DBFE0123237010BD67
:1026A00023B12070BDE81040FFF7F4BE10BD00BF9D
:1026B00082350024014B186D704700BF0040005860
:1026C000084B1A6F120405D41A6F1A671A6F42F476
:1026D00000421A67044A136843F480731360034B83
:1026E00018657047004402580048025800400058DE
:1026F000064A536823F001035360EFF309836833FC
:1027000083F30988002383F31188704730EF00E0DA
:1027100010B5202383F31188104B5B6813F400631A
:1027200018D0F1EE103AEFF309844FF0807344F8BB
:102730004C3C0B4BDB6844F8083CA4F1680383F382
:102740000988FFF733FC18B1064B44F8503C10BD24
:10275000054BFAE783F3118810BD00BF00ED00E0E0
:1027600030EF00E0F3030008F6030008F0B5BFF314
:102770004F8FBFF36F8F1D4B0021C3F85012BFF373
:102780004F8FBFF36F8F5A6942F400325A61BFF323
:102790004F8FBFF36F8FC3F88410BFF34F8FD3F801
:1027A0008020C2F3C904C2F34E325201A50743F69A
:1027B000E07602EA060E284621464EEA0007013975
:1027C000C3F860724F1C00F14040F6D1203A12F17C
:1027D000200FEED1BFF34F8F5A6942F480325A6115
:1027E000BFF34F8FBFF36F8FF0BD00BF00ED00E070
:1027F000FEE70000084A094B09498B4204D3094A05
:102800000021934205D3704752F8040F43F8040B9C
:10281000F3E743F8041BF4E7FC41000850390024B7
:102820005039002450390024D0F8943030B50022BB
:102830009D68D0F8904011464FF0FF3004EB4213F2
:1028400001329542C3F80019C3F81019C3F80809FA
:10285000C3F8001BC3F8101BC3F8080BEED24FF0EF
:102860000113C4F81C3830BD00EB81032DE9F04F93
:10287000D3F80CE0DEF814404F1CD4F800C03F033E
:102880004FEA41186568D0F8902065450AD3D2F820
:102890003438012000FA01F123EA0101C2F83418AA
:1028A000BDE8F08FBEF81060ACEB0503B34228BF63
:1028B000334602EB0806D6F81869B6B2B3EB860FBA
:1028C00013D8A6683A44A6F1040A99465AF804BFF8
:1028D000C2F800B0B9F1040F02D9A9F10409F5E773
:1028E0001E442B44A6606360CCE70020BDE8F08F57
:1028F000890141F02001016103699B06FCD412208B
:1029000000F036BF10B50A4C2046FFF70DF8094B12
:10291000C4F89030084BC4F89430084C2046FFF7B8
:1029200003F8074BC4F89030064BC4F8943010BD40
:10293000843500240000084054400008203600245C
:1029400000000440604000080378012B70B5054684
:102950005DD1494BD0F89040984259D1474BD3F8BC
:10296000D82042F00062C3F8D820D3F8002142F00A
:102970000062C3F80021D3F80021D3F8802042F090
:102980000062C3F88020D3F8802022F00062C3F8F0
:102990008020D3F880300E216520FEF743FC384BB1
:1029A000E360384BC4F800380023C4F8003EC0236D
:1029B0002360D5F890604FF40413A3633369002BB0
:1029C000FCDA012333610C2000F0D2FE3369DB070F
:1029D000FCD4122000F0CCFE3369002BFCDA002678
:1029E000A6602846FFF720FF6B68C4F81068DB6814
:1029F000C4F81468C4F81C68002B3AD1224BA361B8
:102A00004FF0FF336361A36843F00103A36070BD1F
:102A10001E4B9842C8D1194BD3F8D82042F000720F
:102A2000C3F8D820D3F8002142F00072C3F8002187
:102A3000D3F80021D3F8802042F00072C3F8802040
:102A4000D3F8802022F00072C3F88020D3F88020D1
:102A5000D3F8D82022F08062C3F8D820D3F8002120
:102A600022F08062C3F80021D3F800310E214D20FE
:102A700093E7074BC3E700BF8435002400440258A6
:102A80004014004003002002003C30C020360024E7
:102A9000083C30C0F8B5D0F89040054600212046EB
:102AA000FFF726FFD5F8941000234FF001128F682E
:102AB000C4F834384FF00066C4F81C284FF0FF30DB
:102AC00004EB431201339F42C2F80069C2F8006B65
:102AD000C2F80809C2F8080BF2D20B68D5F89020AA
:102AE000C5F89830636210231361166916F010065A
:102AF000FBD1122000F03CFED4F8003823F4FE6332
:102B0000C4F80038A36943F4402343F01003A361E1
:102B10000923C4F81038C4F814380B4BEB604FF09D
:102B2000C043C4F8103B094BC4F8003BC4F810691B
:102B3000C4F80039D5F8983003F1100243F480133B
:102B4000C5F89820A362F8BD30400008408000100E
:102B5000D0F8902090F88A10D2F8003823F4FE6361
:102B600043EA0113C2F80038704700002DE9F04134
:102B70000EB200EB86080D46D8F80C100F6807F06F
:102B80000303022B53D0032B53D03F4A3F4F012B5B
:102B900018BF1746D0F890404FEA451E04EB0E03CD
:102BA0000022C3F8102B8A6905F1100C002A42D0CC
:102BB0004A8A05F158035B013A43E2500123D4F8F5
:102BC0001C2803FA0CF31343A6444A69C4F81C38C2
:102BD0000023CEF8103905F13F03002A3BD00A8AC2
:102BE000898B9208012988BF4A43D0F8981004EBDA
:102BF0008303561841EA0242C0F8986029465A6099
:102C00002046FFF775FED8F80C301B8A43EA85533F
:102C10001F4305F148035B01E7500123D4F81C284A
:102C200003FA05F51543C4F81C58BDE8F081184FA8
:102C3000B0E7184FAEE704EB4613D3F8002B22F4AD
:102C40000042C3F8002BD4F81C28012303FA0CF32C
:102C500022EA0303B8E704EB83030F4A5A6004EB4C
:102C6000461629462046FFF743FED6F8003923F4DE
:102C70000043C6F80039D4F81C38012202FA05F5E1
:102C800023EA0505CFE700BF008000100080041094
:102C90000080081000800C1000040002D0F894207E
:102CA0001268C0F89820FFF7BFBD00005831D0F877
:102CB000903049015B5813F4004004D013F4001F16
:102CC00014BF0120022070474831D0F890304901EC
:102CD0005B5813F4004004D013F4001F14BF01200C
:102CE0000220704700EB8101CB68196A0B68136002
:102CF0004B6853607047000000EB810330B5DD681E
:102D0000AA691368D36019B9402B84BF40231360AC
:102D10006B8A1468D0F890201C44013CB4FBF3F497
:102D20006343033323F0030302EB411043EAC4433C
:102D300043F0C043C0F8103B2B6803F00303012BA2
:102D400009B20ED1D2F8083802EB411013F4807F9B
:102D5000D0F8003B14BF43F0805343F00053C0F859
:102D6000003B02EB4112D2F8003B43F00443C2F8AF
:102D7000003B30BD2DE9F041D0F8906006EB4113E7
:102D80000546D3F8087BC3F8087B3A070C4608D5FC
:102D9000D6F814381B0704D500EB8103DB685B68A9
:102DA0009847FA072FD5D6F81438DB072BD505EB53
:102DB0008403D968CCB98B69488A5E68B6FBF0F2A7
:102DC00000FB12628AB91868DA6890420DD2121AB2
:102DD00083E81400202383F3118821462846FFF757
:102DE0008BFF84F31188BDE8F081012303FA04F21C
:102DF0006B8923EA02036B81CB6823B12146284605
:102E0000BDE8F0411847BDE8F081000000EB810308
:102E100070B5DD68D0F890306C692668E6604A01CC
:102E200056BB1A444FF40020C2F810092A6802F079
:102E30000302012A0AB20ED1D3F8080803EB4214A8
:102E400010F4807FD4F8000914BF40F0805040F0A7
:102E50000050C4F8000903EB4212D2F8000940F018
:102E60000440C2F80009D3F83408012202FA01F143
:102E70000143C3F8341870BD19B9402E84BF4020F7
:102E8000206020682E8A841940F00050013C1A44CA
:102E9000B4FBF6F440EAC440C6E700002DE9F04177
:102EA000D0F8906006EB41130446D3F80879C3F8D4
:102EB0000879FB070D461CD5D6F81038DA0718D567
:102EC00000EB8103D3F80CE0DEF81430D3F800C037
:102ED000DA6894451BD2A2EB0C024FF000081A608E
:102EE000C3F80480202383F31188FFF78FFF88F352
:102EF00011883B0618D5D6F834280123AB4013427D
:102F000012D029462046BDE8F041FFF7ADBC0123B1
:102F100003FA01F2038923EA02030381DEF8083091
:102F2000002BE6D09847E4E7BDE8F0812DE9F047B3
:102F3000D0F890506E69AB691E40F10404466E6192
:102F400003D5BDE8F047FEF769BD002E11DAD5F8CC
:102F5000003E9A071EBFD5F8003E23F00303C5F8D4
:102F6000003ED5F8043823F00103C5F80438FEF715
:102F700085FD330502D52046FEF774FDB7040CD558
:102F8000D5F8083813F0060FEB6823F470530CBF24
:102F900043F4105343F4A053EB60300704D5636847
:102FA000DB680BB120469847F10200F1A180B20224
:102FB0000BD5D4F8908000274FF00109D4F8943055
:102FC0009B68F9B28B4280F0D280F3061AD5D4F810
:102FD00090100A6AC2F30A1702F00F0302F4F0120B
:102FE000B2F5802F00F0EC80B2F5402F0AD104EB4F
:102FF000830301F58051DB68186A00231A469F425B
:1030000040F0D1803003D5F8185835D5E90303D501
:1030100000212046FFF7AEFEAA0303D5012120467A
:10302000FFF7A8FE6B0303D502212046FFF7A2FE9F
:103030002F0303D503212046FFF79CFEE80203D5AA
:1030400004212046FFF796FEA90203D5052120465C
:10305000FFF790FE6A0203D506212046FFF78AFE9D
:103060002B0203D507212046FFF784FEEF0103D58D
:1030700008212046FFF77EFE700340F1C980E90772
:1030800003D500212046FFF709FFAA0703D5012138
:103090002046FFF703FF6B0703D502212046FFF709
:1030A000FDFE2F0703D503212046FFF7F7FEEE06AE
:1030B00003D504212046FFF7F1FEA80603D505211C
:1030C0002046FFF7EBFE690603D506212046FFF7F1
:1030D000E5FE2A0603D507212046FFF7DFFEEB05B4
:1030E00040F1968020460821BDE8F047FFF7D6BEA4
:1030F000D4F890904FF000084FF0010AD4F89430C3
:103100009B685FFA88F7BB42FFF451AF09EB4713A6
:10311000D3F8002902F44022B2F5802F24D1D3F84D
:103120000029002A20DAD3F8002942F09042C3F89F
:103130000029D3F80029002AFBDB3946D4F8900097
:10314000FFF7D6FB22890AFA07F322EA0303238159
:1031500004EB8703DB689B6813B139462046984728
:1031600039462046FFF780FB08F10108C6E708EB67
:103170004112D2F8003B03F44023B3F5802F10D165
:10318000D2F8003B002B0CDA628909FA01F322EA3B
:103190000303638104EB8103DB68DB680BB120462A
:1031A000984701370AE713F0030F08BF0A68072B97
:1031B00098BF027003F101039CBF120A01301EE7A1
:1031C00004EB830301F58051DA6890690268D0F856
:1031D00008C04068A2EB000E00221046974208D1BA
:1031E000DB689B699A683A449A605A6817445F6042
:1031F00008E712F0030F08BF0868964588BF8CF8EF
:10320000000002F1010284BF000A0CF1010CE5E7A5
:10321000BDE8F08708B50348FFF788FEBDE8084021
:10322000FFF776BA8435002408B50348FFF77EFE21
:10323000BDE80840FFF76CBA20360024D0F8903083
:1032400003EB4111D1F8003B43F40013C1F8003BFC
:1032500070470000D0F8903003EB4111D1F80039ED
:1032600043F40013C1F8003970470000D0F89030E3
:1032700003EB4111D1F8003B23F40013C1F8003BEC
:1032800070470000D0F8903003EB4111D1F80039BD
:1032900023F40013C1F800397047000030B5039CD7
:1032A0000172043304FB0325C361049B0363002103
:1032B000059B00604060C1604261026185610462FB
:1032C00042628162C162436330BD00000022416AF4
:1032D00041610161C2608262C2626FF00101FEF76A
:1032E000EDBE000003694269934203D1C2680AB18E
:1032F00000207047181D704703691960C2680132C9
:10330000C260C269134482690361934224BF436A65
:1033100003610021FEF7C6BE38B504460D46E368DA
:103320003BB16269131D1268A3621344E36200207B
:1033300038BD237A33B929462046FEF7A3FE00287C
:10334000EDDA38BD6FF00100FBE70000C368C26929
:10335000013BC3604369134482694361934224BFC4
:10336000436A436100238362036B03B118477047CC
:1033700070B52023044683F31188866A3EB9FFF7AF
:10338000CBFF054618B186F31188284670BDA36AA5
:10339000E26A13F8015BA362934202D32046FFF76F
:1033A000D5FF002383F31188EFE700002DE9F84FE4
:1033B00004460E4690469946202787F3118800253B
:1033C000AA46D4F828B0BBF1000F09D149462046DF
:1033D000FFF7A2FF20B18BF311882846BDE8F88FD4
:1033E000A16AE36AA8EB050B5B1A9B4528BF9B46C5
:1033F000BBF1400F1BD9334601F1400251F8040BD9
:1034000043F8040B9142F9D1A36A40334036A362DA
:103410004035A26AE36A9A4202D32046FFF796FF3C
:103420008AF311884545D8D287F31188C9E7304619
:103430005A46FDF705FDA36A5B445E44A3625D4402
:10344000E7E7000010B5029C0172043303FB04217E
:10345000C36100238362C362039B0363049B006018
:103460004060C46042610261816104624262436300
:1034700010BD0000026AC260426A4261026100221D
:103480008262C2626FF00101FEF718BE43690269F1
:103490009A4203D1C2680AB100207047184650F81A
:1034A000043B0B6070470000C368C2690133C3600E
:1034B0004369134482694361934224BF436A436171
:1034C0000021FEF7EFBD000038B504460D46E36865
:1034D0003BB123691A1DA262E2691344E362002032
:1034E00038BD237A33B929462046FEF7CBFD0028A4
:1034F000EDDA38BD6FF00100FBE7000003691960E9
:10350000C268013AC260C26913448269036193428E
:1035100024BF436A036100238362036B03B118472E
:103520007047000070B5202304460E4683F31188CF
:10353000856A35B91146FFF7C7FF10B185F31188C9
:1035400070BDA36A1E70A36AE26A01339342A3624C
:1035500004D3E16920460439FFF7D0FF002080F34F
:10356000118870BD2DE9F84F04460D4691469A46E4
:103570004FF0200888F311880026B346A76A4FB998
:1035800051462046FFF7A0FF20B187F3118830464F
:10359000BDE8F88FA06AE76AA9EB06033F1A9F42CD
:1035A00028BF1F46402F1BD905F1400355F8042BB7
:1035B00040F8042B9D42F9D1A36A4033A362403600
:1035C000A26AE36A9A4204D3E16920460439FFF70C
:1035D00095FF8BF311884E45D9D288F31188CDE73A
:1035E00029463A46FDF72CFCA36A3B443D44A362BE
:1035F0003E44E5E7026943699A4203D1C3681BB9B7
:10360000184670470023FBE7836A002BF8D0043B81
:103610009B1AF5D01360C368013BC360C3691A44A9
:10362000836902619A4224BF436A03610023836273
:103630000123E5E700F04AB94FF0804300225863C8
:103640001A610222DA6070474FF080430022DA608C
:10365000704700004FF0804358637047FEE700005A
:1036600010B5194CFEF714FCFEF736FD8022174901
:103670002046FEF7BBFC012344F8180C0374144BDE
:10368000144AD96821F4E0610904090C0A4312497B
:10369000DA60CA6842F08072CA60104A1049C2F803
:1036A000B01F116841F0010111601022DA77202269
:1036B00083F82220002383F3118862B60948BDE80D
:1036C0001040FEF7B5BC00BF442E00246C4000083B
:1036D00000ED00E00003FA05F0ED00E0001000E06E
:1036E00055CEACC5744000082DE9F84F1F4C4FF083
:1036F0000008656904F11407C1464FF08043266A4B
:103700005B6AAA689E1B96421DD34FF0200AAA68E6
:10371000236AD5F80CB0134423622B68BB425F6068
:10372000A6EB02066361C5F80C8001D1FFF78CFFA0
:1037300089F311882869D8478AF311886569AB68CD
:103740009E42E4D2D9E76269BA420CD09168236202
:103750008E1B9660A86802282CBF1818981CBDE81C
:10376000F84FFFF777BFBDE8F88F00BF1C2E00248D
:10377000034B59685A68521A9042FBD8704700BFF1
:10378000001000E04B6843608B688360CB68C360C7
:103790000B6943614B6903628B6943620B68036089
:1037A0007047000008B52C4B2C48D3F8882040F215
:1037B000FF710A43C3F88820D3F8882022F4FF62FF
:1037C00022F00702C3F88820D3F88820D3F8E0203D
:1037D0000A43C3F8E020D3F808210A43C3F80821BC
:1037E0001F4AD3F808311146FFF7CCFF1D4802F1FC
:1037F0001C01FFF7C7FF1C4802F13801FFF7C2FFA9
:103800001A4802F15401FFF7BDFF194802F1700197
:10381000FFF7B8FF174802F18C01FFF7B3FF164816
:1038200002F1A801FFF7AEFF144802F1C401FFF74F
:10383000A9FF134802F1E001FFF7A4FF114802F1CC
:10384000FC01FFF79FFF104802F58C71FFF79AFF0C
:10385000BDE8084000F014B90044025800000258C6
:10386000944000080004025800080258000C025856
:10387000001002580014025800180258001C025888
:1038800000200258002402580028025808B500F011
:10389000C5FAFFF7E5FEBDE80840FEF7A7BD00004A
:1038A000704700004FF0804310B51A69920708D5A1
:1038B00000241C61202383F31188FFF715FF84F394
:1038C0001188BDE81040FEF723BF0000134BD3F86A
:1038D000E82042F00102C3F8E820D3F8102142F0BA
:1038E0000102C3F810210E4AD3F81031D36B43F014
:1038F0000103D3634FF080432F229A624FF0FF32CF
:10390000DA6200229A615A63DA605A6001225A61CF
:1039100008211A601C20FDF785BC00BF0044025836
:103920000010005CF8B5514BD3F880204FF0FF3207
:10393000C3F880200024D3F88010C3F88040D3F867
:103940008010D3F88410C3F88420D3F88410C3F80F
:103950008440D3F88410D96F41F0FF4141F4FF0156
:1039600041F4DF4141F07F01D967D96F21F0FF4178
:1039700021F4FF0121F4DF4121F07F01D967D96FE4
:10398000D3F888106FEA41516FEA5151C3F888109B
:10399000D3F88810C1F30A01C3F88810D3F888104F
:1039A000D3F89010C3F89020D3F89010C3F890404B
:1039B000D3F89010D3F89410C3F89420D3F894104F
:1039C000C3F89440D3F89410D3F89810C3F8982013
:1039D000D3F89810C3F89840D3F89810D3F88C1007
:1039E000C3F88C20D3F88C10C3F88C40D3F88C101B
:1039F000D3F89C10C3F89C20D3F89C20C3F89C40BB
:103A0000D3F89C3000F0EAF9194B07229A60194A62
:103A1000DA60194A1A6105225A60184A536A43F457
:103A200080335362C2F88440BFF34F8FD2F88030A6
:103A3000C3F3C904C3F34E335B01A50743F6E07635
:103A400003EA060E284621464EEA00070139C2F86D
:103A500074724F1C00F14040F6D1203B13F1200F4F
:103A6000EED1BFF34F8FBFF36F8FF8BD0044025804
:103A700090ED00E0000004301B00080300ED00E0C2
:103A80005C4B5D4901221A605C4B19609A605C4A8C
:103A9000DA6000221A614FF440429A619A699204F6
:103AA000FCD51A6842F480721A60564B1A6F12F4F1
:103AB000407F1FBF4FF480321A6700221A671A68CE
:103AC00042F001021A604F4A134611684807FCD5BC
:103AD000002111611A6912F03802FBD1012119602D
:103AE0004FF0804159605A67474ADA62474A1A6183
:103AF0001A6842F480321A60424A134611688903F8
:103B0000FCD5116841F0800111601A68D205FCD51E
:103B10003F4A40499A6200225A631963A1F1021197
:103B2000A1F50071DA6399635A643B4A1A643B4A0F
:103B3000DA621A6842F0A8521A60324B1A6802F030
:103B40002852B2F1285FF9D148229A614FF4886275
:103B5000DA6140221A624FF00052DA644FF45001E9
:103B600000221A6559659A652D4A202111601A694B
:103B700042F003021A61234B1A6902F03802182A34
:103B8000FAD1D3F8DC2042F00052C3F8DC20D3F89D
:103B9000042142F00052C3F80421D3F80421D3F8E1
:103BA000DC2042F08042C3F8DC20D3F8042142F04C
:103BB0008042C3F80421D3F80421D3F8DC2042F07A
:103BC0000042C3F8DC20D3F8042142F00042C3F8DD
:103BD0000421D3F80421D3F8F42042F00202C3F800
:103BE000F420D3F81C2142F00202C3F81C21D3F8C0
:103BF0001C3170472004025100C000F000480258F8
:103C000002000001004402580000FF0100889008F3
:103C1000121080000B02030180020101FF07FF0167
:103C200000200052084A08B5936811680B4003F061
:103C30000103936023B1054A13680BB1506898479C
:103C4000BDE80840FEF764BD80000058D03800246D
:103C5000084A08B5936811680B4003F002039360AB
:103C600023B1054A93680BB1D0689847BDE8084076
:103C7000FEF74EBD80000058D0380024084A08B531
:103C8000936811680B4003F00403936023B1054A65
:103C900013690BB150699847BDE80840FEF738BD7D
:103CA00080000058D0380024084A08B5936811688D
:103CB0000B4003F00803936023B1054A93690BB1ED
:103CC000D0699847BDE80840FEF722BD8000005843
:103CD000D0380024084A08B5936811680B4003F0F7
:103CE0001003936023B1054A136A0BB1506A9847D9
:103CF000BDE80840FEF70CBD80000058D038002415
:103D0000174B10B59C681A68144004F478729A60D6
:103D1000A30604D5134A936A0BB1D06A984760068C
:103D200004D5104A136B0BB1506B9847210604D58C
:103D30000C4A936B0BB1D06B9847E20504D5094A46
:103D4000136C0BB1506C9847A30504D5054A936CCE
:103D50000BB1D06C9847BDE81040FEF7D9BC00BF4E
:103D600080000058D03800241A4B10B59C681A689F
:103D7000144004F47C429A60620504D5164A136D1F
:103D80000BB1506D9847230504D5134A936D0BB1C1
:103D9000D06D9847E00404D50F4A136E0BB1506EF6
:103DA0009847A10404D50C4A936E0BB1D06E984786
:103DB000620404D5084A136F0BB1506F984723046F
:103DC00004D5054A936F0BB1D06F9847BDE81040FA
:103DD000FEF79EBC80000058D0380024062108B5AC
:103DE0000846FDF71FFA06210720FDF71BFA0621FA
:103DF0000820FDF717FA06210920FDF713FA06211E
:103E00000A20FDF70FFA06211720FDF70BFA06210D
:103E10002820BDE80840FDF705BA000008B5FFF707
:103E200081FD00F00DF8FDF7A3FBFDF77BFDFDF72D
:103E30004DFCFFF735FDBDE80840FFF7FBBB000078
:103E4000002304491A465A50C8180833802B426090
:103E5000F9D17047D038002410B50139024490429E
:103E600001D1002010BD10F8013B11F8014FA34211
:103E7000F5D0181B10BD0000034611F8012B03F804
:103E8000012B002AF9D170471210121312110000F1
:103E90005C2E0024B029002453544D333248373F60
:103EA0003F3F3F3F00000000009600000000000080
:103EB0000000000000000000000000000000000002
:103EC00000000000391500082515000861150008DC
:103ED0004D15000859150008451500083115000852
:103EE0001D1500086D1500080000000045160008AB
:103EF000311600086D1600085916000865160008EE
:103F0000511600083D16000829160008C9160008B9
:103F1000000000000100000000000000020000009E
:103F20000000000071180008DD1800084000400083
:103F3000F4320024043300240200000000000000DA
:103F4000030000000000000021190008000000002C
:103F500010000000143300240000000001000000E5
:103F600000000000843500240101020025424F4179
:103F7000524425002553455249414C25005069784B
:103F80006861776B3450726F0030313233343536BC
:103F90003738394142434445460000004172647558
:103FA00050696C6F740025424F415244252D424C9C
:103FB000000000008D230008F5210008DD1700082F
:103FC0007123000843000000CC3F000809024300B1
:103FD000020100C0320904000001020201000524B0
:103FE000001001052401000104240202052406003A
:103FF00001070582030800FF09040100020A00000E
:104000000007050102400000070581024000000092
:1040100012000000184000081201100102000040C8
:104020008304405700020102030100000403090455
:1040300000000000911A0008711D00081D1E0008F4
:1040400040004000BC360024BC36002401000000C3
:10405000CC36002480000000400100000800000071
:104060000001000000040000080000006D61696E9E
:10407000000000008C400008D8360024D03800240E
:10408000010000005D3600080000000069646C65F6
:10409000000000000000802A00000000AAAAAAAACE
:1040A00000000000FFFF00000000000000A00A0068
:1040B0000400000000000000AAAAAAAA0000000054
:1040C000FDFF0000000000000000000000500000A4
:1040D00000000000AAAAAAAA000000003FFF0000FA
:1040E00000000000000000000000000000000000D0
:1040F000AAAAAAAA00000000FFFF0000000000001A
:10410000000000000000020000000000AAAAAAAA05
:1041100000000100FFFF0000000000000700000099
:104120000020000000000000AAAAAAAA00100000B7
:10413000FFFF00000000000700000000000000007A
:1041400000000000AAAAAAAA00000000FFFF0000C9
:10415000000000000000000000000000000000005F
:10416000AAAAAAAA00000000FFFF000000000000A9
:10417000000000000000000000000000AAAAAAAA97
:1041800000000000FFFF0000000000000000000031
:104190000000000000000000AAAAAAAA0000000077
:1041A000FFFF000000000000000000000000000011
:1041B00000000000AAAAAAAA00000000FFFF000059
:1041C0000000000000000000FF00000000000000F0
:1041D000983E00083F000000009600000000080024
:1041E000040000002C400008000000000000000057
:1041F00000000000000000000000000000000000BF
:00000001FF
